:020000040000FA
:06000000FEEF32F01200D9
:0600080004EF08F01200F5
:060018000CEF08F01200DD
:06100000FEEF32F01200C9
:06100800CBEF2AF01200FC
:06101800D4EF2AF01200E3
:06102A0002002E6600002A
:10103000940000002000000026660000F802000076
:0410400008000000A4
:0C104400D9CFE6FFE1CFD9FFFB0EDB5057
:1010500029E10201CF51EA6A000FE96E010EEA228E
:101060003C0EEF6ECF29EA6A000FE96E010EEA220C
:10107000FE0EDBCFEFFF020ECF25EA6A000FE96E0E
:10108000010EEA22FD0EDBCFEFFF030ECF25EA6A49
:10109000000FE96E010EEA22FC0EDBCFEFFF040E1B
:1010A000CF273BD00201CF51EA6A000FE96E010E53
:1010B000EA223C0EEF6ECF29EA6A000FE96E010EBC
:1010C000EA22FE0EDBCFEFFF020ECF25EA6A000F09
:1010D000E96E010EEA22FD0EDBCFEFFF030ECF25F6
:1010E000EA6A000FE96E010EEA22FC0EDBCFEFFF89
:1010F000040ECF25EA6A000FE96E010EEA22FB0E0C
:10110000DBCFEFFF050ECF25EA6A000FE96E010E77
:10111000EA223A0EEF6E060ECF27E552E7CFD9FF4F
:101120001200D9CFE6FFE1CFD9FFFE0EDB50410818
:1011300020E1FD0EDB50350A18E0060A13E0010A33
:101140000EE0030A09E0010A04E00001CA0E966FEE
:101150000FD0010EC26E0CD0050EC26E09D0090E62
:10116000C26E06D00D0EC26E03D0110EC26E00D03C
:101170000FD0FE0EDB5042080BE1FD0EDB50320AB1
:1011800004E00001CA0E966F03D0210EC26E00D09B
:10119000E552E7CFD9FF1200D9CFE6FFE1CFD9FF63
:1011A000FE0EDBCFE9FFEA6AE9BEEA68ED0EE9264A
:1011B000020EEA22EF50690A1DE00C0A18E0010A4B
:1011C00013E0070A0EE0010A09E0030A04E0000147
:1011D000CA0E966F12D0010EC26E0FD0050EC26EEF
:1011E0000CD0090EC26E09D00D0EC26E06D0110EC3
:1011F000C26E03D0210EC26E00D0E552E7CFD9FFF8
:101200001200D9CFE6FFE1CFD9FFE652DF6A060E22
:10121000DF24EA6ABB0FE96E020EEA22EF50E66EA7
:10122000DF50EA6AED0FE96E020EEA22E552E7505E
:10123000EF6EDFCFE6FFB0DFE552DF2A060EDF24D8
:10124000EA6ABB0FE96E020EEA22EF50290803E0BA
:10125000070EDF5CDCE3060EDF24EA6ABB0FE96EF3
:10126000020EEA22EF5029080CE1070EDF5C09E2CA
:10127000DF50EA6AED0FE96E020EEA22290EEF6EE8
:1012800003D00001CC0E966FE552E552E7CFD9FFAF
:101290001200D9CFE6FFE1CFD9FF030EE126FD0E04
:1012A000DB500F0BDF6EFD0EDB380F0B0F0BE76E05
:1012B000010EE7CFDBFFFD0EDBCF14F0FE0EDBCF20
:1012C00015F015C014F0156A0F0E1414E76E020E17
:1012D000E7CFDBFFDF50090805E2370EDF2400010E
:1012E000D76F04D0300EDF240001D76F010EDB5022
:1012F000090805E2010EDB50370FD86F04D0010E4C
:10130000DB50300FD86F020EDB50090805E2020EE9
:10131000DB50370FD96F04D0020EDB50300FD96F7E
:10132000FB0EDBCFE9FFEA6AE9BEEA687F0EE92639
:10133000020EEA22FC0EDBCFEFFFFB0EDB28E96E8C
:10134000EA6AE9BEEA687F0EE926020EEA22300E5A
:10135000EF6EFB0EDB50020FE96EEA6AE9BEEA6847
:101360007F0EE926020EEA22D9C0EFFFFB0EDB500A
:10137000030FE96EEA6AE9BEEA687F0EE926020E0B
:10138000EA22D8C0EFFFFB0EDB50040FE96EEA6AD9
:10139000E9BEEA687F0EE926020EEA22D7C0EFFF17
:1013A000FB0EDB50050FE96EEA6AE9BEEA687F0EC4
:1013B000E926020EEA227C0EEF6E030EE15C02E2E9
:1013C000E16AE552E16EE552E7CFD9FF1200D9CFCD
:1013D000E6FFE1CFD9FFFE0EDB50410828E1780E91
:1013E000E66EE66E8050200B01E0010E300FE66ED7
:1013F000780EE66E8050080B01E0010E300FE66EAD
:101400008050040B01E0010E300FE66E8050020B9D
:1014100001E0010E300FE66E8050010B300FE66EDA
:10142000D3EC25F0146E080EE15E145056D0FE0E7B
:10143000DB50420828E1780EE66EE66E8150200B04
:1014400001E0010E300FE66E8150100B01E0010E3D
:10145000300FE66E780EE66E8150040B01E0010E4F
:10146000300FE66E8150020B01E0010E300FE66E88
:101470008150010B300FE66ED3EC25F0146E080E90
:10148000E15E14502AD0FE0EDB50430826E1825064
:10149000800B01E0010E300FE66E8250400B01E040
:1014A000010E300FE66E780EE66EE66EE66E825046
:1014B000040B01E0010E300FE66E8250020B01E0DA
:1014C000010E300FE66E8250010B300FE66ED3EC4A
:1014D00025F0146E080EE15E1450E552E7CFD9FFF7
:1014E0001200D9CFE6FFE1CFD9FFFE0EDB50410855
:1014F00001E0CCD0FD0EDB50350A01E19FD0060A99
:1015000001E17BD0010A52E0030A29E0010A01E06F
:10151000BCD0FC0EDB50300802E180901FD0FC0EE6
:10152000DB50310802E1808019D0FC0EDB506908E5
:1015300007E19280C1500E0802E30F0EC16E0ED07B
:10154000FC0EDB506F0803E19290809007D0FC0EF8
:10155000DB50610803E192800E0EC16E96D0FC0E46
:10156000DB50300802E1809220D0FC0EDB503108C5
:1015700002E180821AD0FC0EDB50690807E19282FA
:10158000C1500D0802E30E0EC16E0FD0FC0EDB50F1
:101590006F0803E19292809208D0FC0EDB50610844
:1015A00004E1030E92120D0EC16E6FD0FC0EDB50E3
:1015B000300802E1809420D0FC0EDB50310802E1BB
:1015C00080841AD0FC0EDB50690807E19284C15078
:1015D0000C0802E30D0EC16E0FD0FC0EDB506F083D
:1015E00003E19294809408D0FC0EDB50610804E182
:1015F000070E92120C0EC16E48D0FC0EDB50300864
:1016000002E180961AD0FC0EDB50690807E1928651
:10161000C1500B0802E30C0EC16E0FD0FC0EDB5064
:101620006F0803E19296809608D0FC0EDB506108AB
:1016300004E10F0E92120B0EC16E27D0FC0EDB5090
:10164000300802E1809A20D0FC0EDB50310802E124
:10165000808A1AD0FC0EDB50690807E1928AC150DB
:101660000A0802E30B0EC16E0FD0FC0EDB506F08B0
:1016700003E1929A809A08D0FC0EDB50610804E1E5
:101680002F0E92120A0EC16E00D013D1FE0EDB5047
:10169000420801E07FD0FD0EDB50350A6EE0010A02
:1016A00060E0060A37E0030A1CE0010A01E071D09D
:1016B000FC0EDB50300802E1819012D0FC0EDB50B2
:1016C000310802E181800CD0FC0EDB50690802E198
:1016D000938006D0FC0EDB506F0802E1939081905E
:1016E00058D0FC0EDB50300802E1819212D0FC0E83
:1016F000DB50310802E181820CD0FC0EDB5069081E
:1017000002E1938206D0FC0EDB506F0802E1939257
:1017100081923FD0FC0EDB50300802E1819420D052
:10172000FC0EDB50310802E181841AD0FC0EDB5044
:10173000690807E19384C150060802E30A0EC16EEE
:101740000FD0FC0EDB506F0803E19394819408D016
:10175000FC0EDB50610804E192689384060EC16EB2
:1017600018D0FC0EDB50300802E1819805D0FC0E49
:10177000DB50310801E181880CD0FC0EDB503008D1
:1017800002E1819A05D0FC0EDB50310801E1818A2B
:1017900000D08FD0FE0EDB50430801E08AD0FD0E52
:1017A000DB50370A6DE0010A52E0040A37E0030A11
:1017B0001CE0010A01E07DD0FC0EDB50300802E1A4
:1017C000829012D0FC0EDB50310802E182800CD0F6
:1017D000FC0EDB50690802E1948006D0FC0EDB5061
:1017E0006F0802E19490829064D0FC0EDB503008C8
:1017F00002E1829212D0FC0EDB50310802E18282BB
:101800000CD0FC0EDB50690802E1948206D0FC0E7D
:10181000DB506F0802E1949282924BD0FC0EDB50B9
:10182000300802E1829412D0FC0EDB50310802E154
:1018300082840CD0FC0EDB50690802E1948406D04F
:10184000FC0EDB506F0802E19494829432D0FC0EBF
:10185000DB50300802E1829C12D0FC0EDB503108D4
:1018600002E1828C0CD0FC0EDB50690802E1948C02
:1018700006D0FC0EDB506F0802E1949C829C19D0CC
:10188000FC0EDB50300802E1829E12D0FC0EDB50D1
:10189000310802E1828E0CD0FC0EDB50690802E1B7
:1018A000948E06D0FC0EDB506F0802E1949E829E5F
:1018B00000D00001A40501E1C188E552E7CFD9FFBE
:1018C0001200D9CFE6FFE1CFD9FF020EE126FE0ECE
:1018D000DB500F0BDF6EFE0EDB380F0B0F0BE76ECE
:1018E000010EE7CFDBFFDF50090805E2370EDF24EA
:1018F0000001D76F04D0300EDF240001D76F010E36
:10190000DB50090805E2010EDB50370FD86F04D019
:10191000010EDB50300FD86FFC0EDBCFE9FFEA6A17
:10192000E9BEEA687F0EE926020EEA22FD0EDBCF51
:10193000EFFFFC0EDB28E96EEA6AE9BEEA687F0E7B
:10194000E926020EEA22780EEF6EFC0EDB50020F43
:10195000E96EEA6AE9BEEA687F0EE926020EEA222B
:10196000780EEF6EFC0EDB50030FE96EEA6AE9BEFB
:10197000EA687F0EE926020EEA22D8C0EFFFFC0ECD
:10198000DB50040FE96EEA6AE9BEEA687F0EE926D9
:10199000020EEA22D7C0EFFFFC0EDB50050FE96E06
:1019A000EA6AE9BEEA687F0EE926020EEA227C0EA8
:1019B000EF6E020EE15C02E2E16AE552E16EE55291
:1019C000E7CFD9FF1200D9CFE6FFE1CFD9FFFD0E57
:1019D000DB50650810E1FE0EDB50320A07E0030A17
:1019E00001E008D094940C0EBD6E04D094920C0EBD
:1019F000BA6E00D011D0FD0EDB5064080DE1FE0E72
:101A0000DB50320A06E0030A01E006D0BD6A948486
:101A100003D0BA6A948200D0E552E7CFD9FF120012
:101A2000D9CFE6FFE1CFD9FFCB50146E156A166A05
:101A3000176A142A000E15221622172214C006F067
:101A400015C007F016C008F017C009F0FA0EDBCF7A
:101A50000BF0FB0EDBCF0CF0FC0EDBCF0DF0FD0E20
:101A6000DBCF0EF052EC31F002C006F003C007F0FD
:101A700004C008F005C009F00B6A010E0C6E0D6A77
:101A80000E6A07EC30F0FA0E06C0DBFFFB0E07C053
:101A9000DBFFFC0E08C0DBFFFD0E09C0DBFFFE0E06
:101AA000DB50320A0EE0030A01E016D0FA0EDBCF5B
:101AB000E6FFFB0EDBCFE6FFB9EC31F0E552E55275
:101AC0000BD0FA0EDBCFE6FFFB0EDBCFE6FF8AEC96
:101AD00031F0E552E55200D0E552E7CFD9FF1200D0
:101AE000D9CFE6FFE1CFD9FFFD0EDBCF14F0FE0E1C
:101AF000DBCF15F0D890155004E62F0E145C000EC5
:101B000015581FE3E00E086E2E0E096EFD0EDBCF9A
:101B10000DF0FE0EDBCF0EF0B4EC2FF008C014F089
:101B200009C015F01406000E155AFD0E14C0DBFF97
:101B3000FE0E15C0DBFF040EE66EBDEC32F0E55282
:101B400075D0FD0EDBCF14F0FE0EDBCF15F0D89074
:101B5000155004E60C0E145C000E15582CE3FD0E17
:101B6000DBCF16F0FE0EDBCF17F0173404E2165071
:101B70002E08000E17541FE3B80E086E0B0E096EE8
:101B8000FD0EDBCF0DF0FE0EDBCF0EF0B4EC2FF030
:101B900008C014F009C015F01406000E155AFD0E09
:101BA00014C0DBFFFE0E15C0DBFF050EE66EBDECBC
:101BB00032F0E5523BD0FD0EDBCF14F0FE0EDBCF52
:101BC00015F0D890155004E6030E145C000E15585D
:101BD0002CE3FD0EDBCF16F0FE0EDBCF17F0173433
:101BE00004E216500B08000E17541FE3EE0E086EA9
:101BF000020E096EFD0EDBCF0DF0FE0EDBCF0EF0F8
:101C0000B4EC2FF008C014F009C015F01406000E53
:101C1000155AFD0E14C0DBFFFE0E15C0DBFF060ECD
:101C2000E66EBDEC32F0E55201D0CB6AFD0EDB5022
:101C3000CB6EE552E7CFD9FF1200D9CFE6FFE1CF57
:101C4000D9FFFE0EDB50380A3EE00F0A36E0010AEB
:101C50002EE0030A26E0010A1EE0070A16E0010A48
:101C60000EE0030A06E0010A01E033D00FEC33F086
:101C700030D0100EE66EA1EC32F0E5522AD0110EF3
:101C8000E66EA1EC32F0E55224D0120EE66EA1EC25
:101C900032F0E5521ED0130EE66EA1EC32F0E552A2
:101CA00018D0140EE66EA1EC32F0E55212D0150EEB
:101CB000E66EA1EC32F0E5520CD0160EE66EA1EC09
:101CC00032F0E55206D0170EE66EA1EC32F0E55286
:101CD00000D0E552E7CFD9FF1200D9CFE6FFE1CF20
:101CE000D9FF060EE126DE6ADE6ADE6ADD6ADD52B3
:101CF000DD52040EDB6A050EDB6AFD0EDBCF14F04D
:101D0000FE0EDBCF15F0166A176A15AE02D0166804
:101D1000176814C0DFFF010E15C0DBFF020E16C0EE
:101D2000DBFF030E17C0DBFFFC0EDB506D0801E08C
:101D3000AFD10201EC97FD0EDBCF17F0FE0EDBCF2B
:101D400018F0196A18BE1968600E146EEA0E156E46
:101D5000166A14C007F015C008F016C009F017C0C5
:101D60000CF018C00DF019C00EF0DAEC2FF007C01F
:101D7000A8F008C0A9F0FD0EDBCF14F0FE0EDBCFFB
:101D800015F0153404E21450F408010E155441E224
:101D9000FD0EDBCF16F0FE0EDBCF17F0173404E29A
:101DA0001650E708030E175434E3170EE66EA1EC45
:101DB00032F0E552D9CFE9FFDACFEAFFEECF06F0F5
:101DC000EECF07F0EECF08F0EFCF09F01B0E0B6E51
:101DD000B70E0C6E0D6A0E6A52EC31F002C006F0BE
:101DE00003C007F004C008F005C009F0E80E0B6E50
:101DF000030E0C6E0D6A0E6AE8EC31F006C0DEFFD1
:101E000007C0DEFF08C0DEFF09C0DDFFDD52DD5286
:101E100009D1FD0EDBCF14F0FE0EDBCF15F015342B
:101E200004E214506408000E155442E2FD0EDBCFAC
:101E300016F0FE0EDBCF17F0173404E21650F4084C
:101E4000010E175435E3160EE66EA1EC32F0E552A2
:101E5000D9CFE9FFDACFEAFFEECF06F0EECF07F0F9
:101E6000EECF08F0EFCF09F0360E0B6E6E0E0C6E53
:101E7000010E0D6E0E6A52EC31F002C006F003C086
:101E800007F004C008F005C009F0E80E0B6E030E61
:101E90000C6E0D6A0E6AE8EC31F006C0DEFF07C07A
:101EA000DEFF08C0DEFF09C0DDFFDD52DD52BAD023
:101EB000FD0EDBCF14F0FE0EDBCF15F0153404E27F
:101EC00014503208000E155431E2FD0EDBCF16F02F
:101ED000FE0EDBCF17F0173404E216506408000E34
:101EE000175424E3140EE66EA1EC32F0E552D9CF7C
:101EF000E9FFDACFEAFFEECF06F0EECF07F0EECF44
:101F000008F0EFCF09F0770E0B6E010E0C6E0D6A24
:101F10000E6A52EC31F002C0DEFF03C0DEFF04C0E7
:101F2000DEFF05C0DDFFDD52DD527CD0FD0EDBCFD4
:101F300014F0FE0EDBCF15F0153404E214500A083D
:101F4000000E155431E2FD0EDBCF16F0FE0EDBCF96
:101F500017F0173404E216503208000E175424E329
:101F6000130EE66EA1EC32F0E552D9CFE9FFDACFDD
:101F7000EAFFEECF06F0EECF07F0EECF08F0EFCF9E
:101F800009F0EE0E0B6E020E0C6E0D6A0E6A52EC2C
:101F900031F002C0DEFF03C0DEFF04C0DEFF05C07B
:101FA000DDFFDD52DD523ED0FD0EDBCF14F0FE0E24
:101FB000DBCF15F0D890155004E6010E145C000E2E
:101FC000155830E3FD0EDBCF16F0FE0EDBCF17F019
:101FD000173404E216500A08000E175423E3100EBB
:101FE000E66EA1EC32F0E552D9CFE9FFDACFEAFF95
:101FF000EECF06F0EECF07F0EECF08F0EFCF09F00E
:10200000700E0B6E170E0C6E0D6A0E6A52EC31F0EC
:1020100002C0DEFF03C0DEFF04C0DEFF05C0DDFF3F
:10202000DD52DD52176A186A010E196EDFCF1AF001
:10203000DBCF1BF01C6A1BBE1C681A50175C146EA9
:102040001B501858156E1C501958166E190E142670
:10205000000E15221622040E14C0DBFF050E15C05B
:10206000DBFFF294040EDBCFE6FF050EDBCFE6FFCD
:1020700085EC32F0E552E552040EDBCF14F0050E8C
:10208000DBCF15F014C0F3FF15C0F4FF9ED09DD038
:10209000FC0EDB50750801E095D00201EC870001D1
:1020A000E80EAA6F030EAB6FFD0EDBCF17F0FE0E2E
:1020B000DBCF18F0196A18BE1968600E146EEA0EAC
:1020C000156E166A14C007F015C008F016C009F0A6
:1020D00017C00CF018C00DF019C00EF0DAEC2FF09C
:1020E00007C0A8F008C0A9F0FD0EDBCF14F0FE0E6B
:1020F000DBCF15F0D890155004E6010E145C000EED
:1021000015582FE3FD0EDBCF16F0FE0EDBCF17F0D8
:10211000173404E21650E708030E175422E3100E9A
:10212000E66EA1EC32F0E552D9CFE9FFDACFEAFF53
:10213000EECF06F0EECF07F0EECF08F0EFCF09F0CC
:10214000060E0B6E0C6A0D6A0E6A52EC31F002C07C
:10215000DEFF03C0DEFF04C0DEFF05C0DDFFDD5291
:10216000DD52176A186A010E196EDFCF1AF0DBCF45
:102170001BF01C6A1BBE1C681A50175C146E1B50A7
:102180001858156E1C501958166E040E14C0DBFF3B
:10219000050E15C0DBFFF294040EDBCFE6FF050E43
:1021A000DBCFE6FF85EC32F0E552E552040EDBCFE3
:1021B00014F0050EDBCF15F014C0F3FF15C0F4FFCB
:1021C00004D003D00001CB0E966F060EE15C02E254
:1021D000E16AE552E16EE552E7CFD9FF1200D9CFAF
:1021E000E6FFE1CFD9FFFE0EDB50340A1EE0070AFE
:1021F00016E0010A0EE0030A06E0010A01E01BD026
:102200000CEC33F018D04D0EE66E0CEC32F0E552CB
:1022100012D05D0EE66E0CEC32F0E5520CD06D0E75
:10222000E66E0CEC32F0E55206D07D0EE66E0CEC5C
:1022300032F0E55200D0E552E7CFD9FF1200D9CFF6
:10224000E6FFE1CFD9FF060EE126DE6ADE6ADE6A2E
:10225000DD6ADD52DD52040EDB6A050EDB6AFD0E1F
:10226000DBCF14F0FE0EDBCF15F0166A176A15AE41
:1022700002D01668176814C0DFFF010E15C0DBFF1F
:10228000020E16C0DBFF030E17C0DBFFFC0EDB5097
:102290006D0801E029D1FD0EDBCF14F0FE0EDBCF7F
:1022A00015F0153404E214501408000E155431E2F0
:1022B000FD0EDBCF16F0FE0EDBCF17F0173404E275
:1022C00016502808000E175424E37D0EE66E0CEC21
:1022D00032F0E552D9CFE9FFDACFEAFFEECF06F0D0
:1022E000EECF07F0EECF08F0EFCF09F0DC0E0B6E6B
:1022F000050E0C6E0D6A0E6A52EC31F002C0DEFF64
:1023000003C0DEFF04C0DEFF05C0DDFFDD52DD528D
:10231000BAD0FD0EDBCF14F0FE0EDBCF15F0153476
:1023200004E214500A08000E155431E2FD0EDBCF12
:1023300016F0FE0EDBCF17F0173404E21650140827
:10234000000E175424E36D0EE66E0CEC32F0E552ED
:10235000D9CFE9FFDACFEAFFEECF06F0EECF07F0F4
:10236000EECF08F0EFCF09F0B80E0B6E0B0E0C6E2F
:102370000D6A0E6A52EC31F002C0DEFF03C0DEFFD0
:1023800004C0DEFF05C0DDFFDD52DD527CD0FD0E56
:10239000DBCF14F0FE0EDBCF15F0153404E2145041
:1023A0000508000E155431E2FD0EDBCF16F0FE0ECF
:1023B000DBCF17F0173404E216500A08000E17544A
:1023C00024E35D0EE66E0CEC32F0E552D9CFE9FF66
:1023D000DACFEAFFEECF06F0EECF07F0EECF08F04F
:1023E000EFCF09F0700E0B6E170E0C6E0D6A0E6AB1
:1023F00052EC31F002C0DEFF03C0DEFF04C0DEFF9E
:1024000005C0DDFFDD52DD523ED0FD0EDBCF14F006
:10241000FE0EDBCF15F0D890155004E6010E145CCB
:10242000000E155830E3FD0EDBCF16F0FE0EDBCFAD
:1024300017F0173404E216500508000E175423E372
:102440004D0EE66E0CEC32F0E552D9CFE9FFDACF53
:10245000EAFFEECF06F0EECF07F0EECF08F0EFCFB9
:1024600009F0E00E0B6E2E0E0C6E0D6A0E6A52EC29
:1024700031F002C0DEFF03C0DEFF04C0DEFF05C096
:10248000DDFFDD52DD52176A186A010E196EDFCFCB
:102490001AF0DBCF1BF01C6A1BBE1C681A50175CBD
:1024A000146E1B501858156E1C501958166E040ED9
:1024B00014C0DBFF050E15C0DBFF9E90040EDBCFC2
:1024C000E6FF050EDBCFE6FF69EC32F0E552E552A0
:1024D000040EDBCF14F0050EDBCF15F014C0F3FFB4
:1024E00015C0F4FF76D075D0FC0EDB5075086EE198
:1024F000FD0EDBCF14F0FE0EDBCF15F0D89015509B
:1025000004E6010E145C000E15582FE3FD0EDBCF20
:1025100016F0FE0EDBCF17F0173404E21650E70872
:10252000030E175422E34D0EE66E0CEC32F0E5522A
:10253000D9CFE9FFDACFEAFFEECF06F0EECF07F012
:10254000EECF08F0EFCF09F00C0E0B6E0C6A0D6A9F
:102550000E6A52EC31F002C0DEFF03C0DEFF04C0A1
:10256000DEFF05C0DDFFDD52DD52176A186A010E7D
:10257000196EDFCF1AF0DBCF1BF01C6A1BBE1C6884
:102580001A50175C146E1B501858156E1C501958B1
:10259000166E040E14C0DBFF050E15C0DBFF9E9007
:1025A000040EDBCFE6FF050EDBCFE6FF69EC32F071
:1025B000E552E552040EDBCF14F0050EDBCF15F02B
:1025C00014C0F3FF15C0F4FF04D003D00001CB0EFC
:1025D000966F060EE15C02E2E16AE552E16EE552B9
:1025E000E7CFD9FF1200D9CFE6FFE1CFD9FF040E24
:1025F000E126DF6A010EDB6A020EDB6A030EDB6A8C
:102600005A0E0201BC5D1DE14D0EBD5D19E1440E87
:10261000BE5D16E1310EE66E760EE66E320EE66EA9
:10262000310EE66E500EE66E430EE66E690EE66EF5
:102630003A0EE66ED3EC25F0146E080EE15E1450EF
:10264000AAD04D0EBC5D1BE1440EBD5D08E1490EF4
:10265000BE5D05E10F0EC16E926893680FD0410E0A
:10266000BD5D0CE14E0EBE5D09E19268040E936EF5
:10267000010EC26E060EC16EBF0EC06E8CD0440E2F
:10268000BC5D01E088D0500EBD5D2BE1410EBE5D0A
:1026900028E1780EE66EE66E8050200B01E0010E18
:1026A000300FE66E780EE66E8050080B01E0010EEA
:1026B000300FE66E8050040B01E0010E300FE66E25
:1026C0008050020B01E0010E300FE66E8050010BCE
:1026D000300FE66ED3EC25F0146E080EE15E145058
:1026E0005AD0500EBD5D2BE1420EBE5D28E1780E42
:1026F000E66EE66E8150200B01E0010E300FE66EB3
:102700008150100B01E0010E300FE66E780EE66E80
:102710008150040B01E0010E300FE66E8150020B78
:1027200001E0010E300FE66E8150010B300FE66EB6
:10273000D3EC25F0146E080EE15E14502CD0500E30
:10274000BD5D29E1430EBE5D26E18250800B01E0B4
:10275000010E300FE66E8250400B01E0010E300F8B
:10276000E66E780EE66EE66EE66E8250040B01E0D1
:10277000010E300FE66E8250020B01E0010E300FA9
:10278000E66E8250010B300FE66ED3EC25F0146E2E
:10279000080EE15E1450020E0001965D02E1020196
:1027A000BF6B040EE15C02E2E16AE552E16EE552C4
:1027B000E7CFD9FF1200D9CFE6FFE1CFD9FFE6522C
:1027C000F250800B01E0010EDF6EF29EA69EA69CE9
:1027D000A684FE0EDB50A96EFD0EDB50A86E550ED2
:1027E000A76EAA0EA76EA682A6B2FED7A694DF5049
:1027F000E8B0F28EE8A0F29EE552E552E7CFD9FFAD
:102800001200D9CFE6FFE1CFD9FFA69CA69EFE0E0F
:10281000DB50A96EA680A85000D0E552E7CFD9FFC3
:102820001200D9CFE6FFE1CFD9FFE652FB0EDB5015
:10283000F66EFC0EDB50F76EFD0EDB50F86EE00E10
:10284000F616DF6ADFCF14F03F0EE76E1418E8AE1D
:1028500002D0143403D0E750D880145412E3090096
:10286000DFCF14F0156A14BE1568F90EDB5014247E
:10287000E96EFA0EDB501520EA6EF5CFEFFFDF2A86
:10288000E1D7E552E552E7CFD9FF1200D9CFE6FFF5
:10289000E1CFD9FFE652A6B2FED7F29CF29EFD0E22
:1028A000DB50F86EFC0EDB50F76EFB0EDB50F66E65
:1028B000E00EF616A68EA69CA684A688550EA76ED8
:1028C000AA0EA76EA6820000F90EDBCF14F0FA0E56
:1028D000DBCF15F015C014F0156A1450EA6EFF0E28
:1028E000E76EF90EDBCF14F0FA0EDBCF15F0E750F0
:1028F0001416156A1450E96E0A00200EDF6EDF50C0
:1029000005E0EE50F56E0F00DF06F9D7A68EA69C07
:10291000A684550EA76EAA0EA76EA6820000200EF2
:10292000DF6EDF5005E0EE50F56E0F00DF06F9D7E1
:10293000A68EA69CA684550EA76EAA0EA76EA6828A
:102940000000A694F28EF28CE552E552E7CFD9FF53
:102950001200550EA76EAA0EA76EA682A6B2FED7CB
:10296000A6941200D9CFE6FFE1CFD9FFF29CF29EE8
:10297000FD0EDB50F86EFC0EDB50F76EFB0EDB50ED
:10298000F66E0001DC6B0E0E0001DC5D17E200014B
:10299000DC51E76EF90EDBCFE9FFFA0EDBCFEAFF81
:1029A000E750E926000EEA22EF50F56E0C00C40E47
:1029B000A66ECFDF09000001DC2BE5D7F28EF28C8A
:0829C000E552E7CFD9FF120038
:0829C800D9CFE6FFE1CFD9FFF2
:1029D000E652A09A6A6A686A706A020EE66EE66A51
:1029E000E66A710EE66E0F0EE66E38EC31F0146E8C
:1029F000050EE15E1450160E6F6E9F0E6B6E7B0E11
:102A0000696EDF6ADF50146E156A0C0E145C000EDE
:102A1000155810E2DF50040DF3CFE9FFF4CFEAFFC1
:102A2000000EE926040EEA22EE6AEE6AEE6AEE6A0B
:102A3000DF2AE8D76D8C6E6A6D986D9C68A607D00A
:102A400068960001776B7C6B7D6B7E6BF7D700011E
:102A5000010E906F916F926B936B846BDF6A030E24
:102A6000DF5C26E2EA6ADF34FE0BEA36E96E6D0EC1
:102A7000E926000EEA22EE6AED6AEA6ADF34FE0B0E
:102A8000EA36E96E670EE926000EEA22EE6AED6A82
:102A9000DF50EA6A880FE96E000EEA22EF6ADF5023
:102AA000EA6A8B0FE96E000EEA22EF6ADF2AD7D7B7
:102AB0000001080E6D6F040E6E6F160E706E04012D
:102AC000300E026F040E036F080E016F840E006F4C
:102AD0000001616B606BE552E552E7CFD9FF120050
:102AE000D9CFE6FFE1CFD9FFE6520001605116E1F0
:102AF00006D06D6A696A0001606BA19AB9D06D6AEF
:102B0000696A160E6F6E9F0E6B6E7B0E696E6DB6E8
:102B100002D06D86FCD70001010E606F600508E1F0
:102B20006DBA06D0686A696A69806988020E606F4A
:102B30006850040B05E06950040B02E06894CBD8A0
:102B40006DA202D0A19A94D06850010B08E06950A0
:102B5000010B05E039DF0001040E606F68906850DA
:102B6000100B05E06950100B02E0A0D8689868AC23
:102B700019D069AC0FD0010EE66EE66A000EE66E63
:102B8000E66A730EE66EE66A3BEC2DF0146E060EF6
:102B9000E15E1450689C00018E5101E08E078E5159
:102BA00001E165DB6850200B04E06950200B01E077
:102BB00064D86850020B13E06950020B10E0010E5C
:102BC000E66EE66A000EE66EE66AE6687F0EE66E80
:102BD0003BEC2DF0146E060EE15E14506A6A040E92
:102BE0000001E76E6019E8AE02D0E73402D0E7508A
:102BF000605D02E2A19A3CD069A639D0DF6A040E7A
:102C0000DF5C35E268A630D06CCF85F000018551DD
:102C1000780BE842E842E842866F689685B508D0AE
:102C20008651EA6A8B0FE96E000EEA22EF7007D038
:102C30008651EA6A880FE96E000EEA22EF7086512B
:102C400002E160D810D0000EE66EE66A850EE66EF0
:102C5000000EE66E720EE66EE66A3BEC2DF0146E28
:102C6000060EE15E145001D002D0DF2AC8D7A19A27
:102C7000E552E552E7CFD9FF120070A015D063C02E
:102C8000E9FF64C0EAFFEF5080080DE16DC0E9FF85
:102C90006EC0EAFFEF50840806E163C0E9FF64C03C
:102CA000EAFF8C0EEF6E7090689A12006984689843
:102CB0006D820001010E846F000EE66EE66AE66E1C
:102CC000E66A750EE66EE66A3BEC2DF0146E060EB3
:102CD000E15E145012000001846B000EE66EE66A9D
:102CE000E66EE66A740EE66EE66A3BEC2DF0146E54
:102CF000060EE15E14506D92699468A402D0689447
:102D0000FCD71200D9CFE6FFE1CFD9FFE652000190
:102D10002D0E8E6FFD0E851553E17E0E8515E84054
:102D20007F0B040DF3CF63F0F4CF64F0000E632744
:102D3000040E642363C065F064C066F0657563C00B
:102D4000E9FF64C0EAFFEF503C0BE842E8420D089F
:102D500035E1DF6A080EDF5C23E263C0E9FF64C08F
:102D6000EAFF020EE926000EEA22EE50EFCFEAFF5C
:102D7000E96EEF50E66EDF50EA6A300FE96E040E3E
:102D8000EA22E552E750EF6E63C0E9FF64C0EAFF54
:102D9000020EE926000EEA22EE2AEF22DF2ADAD717
:102DA00063C0E9FF64C0EAFF020EE926000EEA22D2
:102DB000300EEE6E040EED6E0DD801D03AD805D06F
:102DC000FD0E8515040801E15AD8E552E552E7CF1A
:102DD000D9FF12000001736B8F6B926B936B876B43
:102DE000746B6DC0E9FF6EC0EAFFEF9E6D756DC03C
:102DF000E9FF6EC0EAFFEF9E6D7565C0E9FF66C032
:102E0000EAFFEF9E776B786B796B7C6B7D6B7E6BEB
:102E100090D8000EE66EE66AE66EE66A030EE66E8F
:102E2000E66A3BEC2DF0146E060EE15E145089EF5D
:102E30001AF0020E0001745D03E14CEC1BF01ED091
:102E4000746B87511AE165C0E9FF66C0EAFFEE5274
:102E5000080EEF6E65C0E9FF66C0EAFF020EE926C4
:102E6000000EEA22300EEE6E040EED6E65C0E9FF34
:102E700066C0EAFF8C0EEF6E01D0876B1200D9CFCF
:102E8000E6FFE1CFD9FFE6526DC0E9FF6EC0EAFF71
:102E9000EF50400B01E0010EDF6E00016D75080E72
:102EA000605D09E132C46EFF6E5003E0100E606F8A
:102EB00002D0040E606F740528E16DC0E9FF6EC09A
:102EC000EAFF020EE926000EEA22380EEE6E040E2C
:102ED000ED6E80DB020E0001735D07E16DC0E9FF5E
:102EE0006EC0EAFF840EEF6E0FD0DF5007E16DC0B9
:102EF000E9FF6EC0EAFFC80EEF6E06D06DC0E9FFB5
:102F00006EC0EAFF880EEF6E0FD07CAF0CD07F5101
:102F1000801107E005D080C0FAFF00017F51F96EF3
:102F2000FADF00017C9F746BE552E552E7CFD9FFD1
:102F3000120004013051600BE842E842E842E842E6
:102F4000E842000901E059D031510C0A55E00B0A62
:102F500044E00C0A36E0010A27E00B0A23E0020AEB
:102F600021E0030A1DE0080A11E0010A0CE00F0A43
:102F700008E0030A01E040D00001778F080E606F7F
:102F80003CD006DA3AD0ECEC1BF037D00001610EF1
:102F9000756F000E766F7781010E786F778F2DD069
:102FA00057DA2BD02BD829D034510001756F766BAE
:102FB000620E7527000E76237781010E786F778F6A
:102FC0001CD00001778F04013451EA6A620FE96E68
:102FD000000EEA2232C4EFFF10D0000EE66EE66A61
:102FE000E66EE66A020EE66EE66A3BEC2DF0146EC3
:102FF000060EE15E145001D000D01200D9CFE6FFDA
:10300000E1CFD9FF030EE1260401320510E1305172
:103010001F0B00090CE10001778F030E0401315DE5
:1030200004E10001010E836F02D00001836B0401F3
:10303000325101E012D130511F0B020801E00DD1D5
:1030400034510F0B000901E108D134510F0B020874
:1030500001E203D1200E0001605D01E0FED0778F18
:10306000040134BF1AD034510F0BE96EEA6AD890CC
:10307000E936EA36670EE926000EEA22EECFDEFFD9
:10308000EDCFDDFF34510F0BEA6A8B0FE96E000EB6
:10309000EA22020EEFCFDBFF19D034510F0BE96E9D
:1030A000EA6AD890E936EA366D0EE926000EEA2281
:1030B000EECFDEFFEDCFDDFF34510F0BEA6A880F54
:1030C000E96E000EEA22020EEFCFDBFFD950020FAD
:1030D000E96EDACFEAFFEF50010B03E1000EDF9457
:1030E00001D0DF8434BF10D034510F0BE96EEA6A8F
:1030F000D890E936EA36670EE926000EEA22DECFDE
:10310000EEFFDDCFEDFF0FD034510F0BE96EEA6A11
:10311000D890E936EA366D0EE926000EEA22DECFB7
:10312000EEFFDDCFEDFF030E315D23E1DECFE9FFE2
:10313000DDCFEAFFEF50800B13E034BF09D03451EC
:103140000F0BEA6A8B0FE96E000EEA22EF8208D0BD
:1031500034510F0BEA6A880FE96E000EEA22EF8203
:10316000840E146EDECFE9FFDDCFEAFF1450EF12BC
:1031700074D0DF74DECFE9FFDDCFEAFFEF50800BC4
:103180001BE0DECFE9FFDDCFEAFFEF9EDECFE9FFF8
:10319000DDCFEAFFEF8C020EE66EE66ADECFE6FFD9
:1031A000DDCFE6FF050EE66EE66A3BEC2DF0146E11
:1031B000060EE15E145005D0DECFE9FFDDCFEAFF59
:1031C000EF8CDF74D950020FE96EDACFEAFFEF50CF
:1031D000020B0EE1DECFE9FFDDCFEAFFEF50800BFF
:1031E00034E0DECFE9FFDDCFEAFFEF50040B2DE145
:1031F000040134BF09D034510F0BEA6A8B0FE96E1A
:10320000000EEA22EF9208D034510F0BEA6A880FC1
:10321000E96E000EEA22EF923B0E146EDECFE9FF5C
:10322000DDCFEAFF1450EF16020EE66EE66ADECF3F
:10323000E6FFDDCFE6FF050EE66EE66A3BEC2DF01D
:10324000146E060EE15E145008D03B0E146EDECFF5
:10325000E9FFDDCFEAFF1450EF16030EE15C02E256
:10326000E16AE552E16EE552E7CFD9FF12000001B5
:1032700090514DE1010E906F915149E1010E916F16
:10328000020E745D0DE16DC0E9FF6EC0EAFFEE5203
:10329000EF6A6DC0E9FF6EC0EAFFC80EEF6E37D06F
:1032A000740535E1876B63C0E9FF64C0EAFFEE5245
:1032B000080EEF6E63C0E9FF64C0EAFF020EE92664
:1032C000000EEA22300EEE6E040EED6E63C0E9FFD2
:1032D00064C0EAFF840EEF6E010E876F65C0E9FFE0
:1032E00066C0EAFFEE52080EEF6E65C0E9FF66C0E9
:1032F000EAFF020EE926000EEA22300EEE6E040E00
:10330000ED6E65C0E9FF66C0EAFF800EEF6E120049
:103310000001926B936B020E745D1AE165C0E9FFC8
:1033200066C0EAFFEE52080EEF6E65C0E9FF66C0A8
:10333000EAFF020EE926000EEA22380EEE6E040EB7
:10334000ED6E65C0E9FF66C0EAFFC80EEF6E1FD0E4
:1033500078510401365D000179510401375904E2C6
:1033600036C478F037C479F035D96DC0E9FF6EC046
:10337000EAFF020EE926000EEA22380EEE6E040E77
:10338000ED6E6DC0E9FF6EC0EAFFC80EEF6E120071
:10339000800E0401305D5BE10001C00E776F040117
:1033A0003351030A34E0010A0EE0030A03E000018E
:1033B000776B4DD00001B20E756F600E766F120EF6
:1033C000786F796B44D03251F66EF76AD890F63642
:1033D000F736730EF626610EF7220900F5CF75F069
:1033E0000A00F5CF76F0020E0001F76A7525F66E39
:1033F0007651F7220800F5CF78F0030EF76A7525AD
:10340000F66E7651F7220800F5CF79F020D0030E42
:10341000325D1AE23251F66EF76AD890F636F73618
:10342000750EF626610EF7220900F5CF75F00A0039
:10343000F5CF76F075C0F6FF76C0F7FF0800F550BF
:103440000001786F796B02D00001776B00D0120019
:10345000D9CFE6FFE1CFD9FF020EE1260401386B98
:10346000396B30511F0B020A12E0030A0DE0010A0A
:1034700001E03BD00001778F040138810001830512
:1034800002E10401388331D00001778F2ED0000192
:10349000778F040134BF10D034510F0BE96EEA6A04
:1034A000D890E936EA36670EE926000EEA22EECF1A
:1034B000DEFFEDCFDDFF0FD034510F0BE96EEA6A6E
:1034C000D890E936EA366D0EE926000EEA22EECFF4
:1034D000DEFFEDCFDDFFDECFE9FFDDCFEAFFEF500E
:1034E000040B02E0010E386F00D0000177AF07D067
:1034F000380E756F040E766F7781020E786F020EAC
:10350000E15C02E2E16AE552E16EE552E7CFD9FF04
:1035100012006D98000177BF2BD07CAF09D0020E4E
:10352000746F935101E1F4DE0001916B906B1FD039
:1035300065C0E9FF66C0EAFFEE52080EEF6E65C097
:10354000E9FF66C0EAFF020EE926000EEA22300E0D
:10355000EE6E040EED6E65C0E9FF66C0EAFF8C0EEC
:10356000EF6E6DC0E9FF6EC0EAFF840EEF6E31D0E2
:10357000040130AF0DD00001010E746F925101E1D2
:10358000C7DE0001916B906B8F5101E170DE21D09D
:103590000001020E746F65C0E9FF66C0EAFFEE52DB
:1035A000080EEF6E65C0E9FF66C0EAFF020EE9266D
:1035B000000EEA22300EEE6E040EED6E65C0E9FFDD
:1035C00066C0EAFF840EEF6E916B906B8F5101E144
:1035D0004EDE1200D9CFE6FFE1CFD9FFE652080E4A
:1035E000DF6E0001785D000E79590BE278C0DFFFD5
:1035F000735103E1010E736F04D0730502E1020EF3
:10360000736FDF50146E156A1450785D786F155023
:103610007959796F6DC0E9FF6EC0EAFFEE52DFCFD6
:10362000EFFF380E816F040E826F77B119D0DF5033
:1036300016E075C0F6FF76C0F7FF752B000E7623F7
:103640000800F550E66E81C0E9FF82C0EAFF812BD9
:10365000000E8223E552E750EF6EDF06E8D717D061
:10366000DF5015E075C0E9FF76C0EAFF752B000E4C
:103670007623EF50E66E81C0E9FF82C0EAFF812B1E
:10368000000E8223E552E750EF6EDF06E9D7E552E0
:10369000E552E7CFD9FF1200D9CFE6FFE1CFD9FF3E
:1036A000020EE12663C0E9FF64C0EAFFEE52EFCFED
:1036B000DFFFDFCF14F0145000017D5D000E7E5956
:1036C00002E27DC0DFFFDF50146E156A14507D5D8D
:1036D0007D6F15507E597E6F010EDB6ADF50F36EF1
:1036E000010EDBCFF4FFF350F45C16E2010EDB5069
:1036F000EA6A380FE96E040EEA22EF50E66E7AC0ED
:10370000E9FF7BC0EAFF7A2B000E7B23E552E750EE
:10371000EF6E010EDB2AE2D7000ED8807D55000E39
:103720007E5528E265C0E9FF66C0EAFFEE52080E4A
:10373000EF6E65C0E9FF66C0EAFF020EE926000EE3
:10374000EA22380EEE6E040EED6E63C0E9FF64C02F
:10375000EAFFEF50400B07E165C0E9FF66C0EAFFF2
:10376000C80EEF6E06D065C0E9FF66C0EAFF880E9E
:10377000EF6E28D065C0E9FF66C0EAFFEE52080E82
:10378000EF6E65C0E9FF66C0EAFF020EE926000E93
:10379000EA22300EEE6E040EED6E65C0E9FF66C0E3
:1037A000EAFF840EEF6E7F51801107E005D080C0E4
:1037B000FAFF00017F51F96EFADF00017C9F8F5103
:1037C00001E155DD020EE15C02E2E16AE552E16EE3
:1037D000E552E7CFD9FF1200D9CFE6FFE1CFD9FFFD
:1037E000E6520001778F020EE66EE66AE66A710E17
:1037F000E66E0F0EE66E38EC31F0146E050EE15EEB
:103800001450DF6ADF50146E156A0C0E145C000E43
:10381000155810E2DF50040DF3CFE9FFF4CFEAFFB3
:10382000000EE926040EEA22EE6AEE6AEE6AEE6AFD
:10383000DF2AE8D76D8C010EE66EE66AE66A620E54
:10384000E66E000EE66E38EC31F0146E050EE15EA9
:1038500014506D9C0001080E6D6F040E6E6F000E0B
:10386000636F040E646F63C065F064C066F032C4B9
:1038700061F0615103E1100E606F13D0010EE66E2E
:10388000E66A610EE66E000EE66E010EE66EE66A10
:103890003BEC2DF0146E060EE15E14500001200E7C
:1038A000606FE552E552E7CFD9FF1200D9CFE6FFAE
:1038B000E1CFD9FF020EE126000EDE6E040EDD6EB2
:1038C000FD0EDB50E824166EFE0EDB50040DF350A7
:1038D0001624040DF3CF14F0F4CF15F0D9CFE9FF7F
:1038E000DACFEAFF1450EE261550ED22DECFE9FFC5
:1038F000DDCFEAFFEF9EFD0EDB500FE1FE0EEA6A20
:10390000DB34FE0BEA36E96E670EE926000EEA228A
:10391000DECFEEFFDDCFEDFF0ED0FE0EEA6ADB3428
:10392000FE0BEA36E96E6D0EE926000EEA22DECFC6
:10393000EEFFDDCFEDFFDECFE9FFDDCFEAFFEF9C4D
:10394000DECFE9FFDDCFEAFF040EE926000EEA2212
:10395000EF8C020EE15C02E2E16AE552E16EE552B3
:10396000E7CFD9FF1200D9CFE6FFE1CFD9FF020E92
:10397000E126FD0EDBA407D0E66AFE0EDBCFE6FFF4
:1039800095DFE552E552FD0EDBA208D0010EE66E92
:10399000FE0EDBCFE6FF8ADFE552E552FE0EDB507E
:1039A000156A700F146E0F0E152214C0DEFF15C0BD
:1039B000DDFFDECFE9FFDDCFEAFFFD0EDBCFEFFF5E
:1039C000020EE15C02E2E16AE552E16EE552E7CF08
:1039D000D9FF1200D9CFE6FFE1CFD9FF020EE126D1
:1039E000FE0EDB5020E165C0E9FF66C0EAFFEE5243
:1039F000080EEF6E65C0E9FF66C0EAFF020EE92619
:103A0000000EEA22300EEE6E040EED6E65C0E9FF88
:103A100066C0EAFF8C0EEF6E6DC0E9FF6EC0EAFF74
:103A2000840EEF6E3DD0FD0EDB50E824166EFE0EC8
:103A3000DB50040DF3501624040DF3CF14F0F4CF33
:103A400015F0000E1426040E152214C0DEFF15C05A
:103A5000DDFF840E146EDECFE9FFDDCFEAFF1450E8
:103A6000EF12FD0EDB50E824166EFE0EDB50040D47
:103A7000F3501624010F040DF3CF14F0F4CF15F01A
:103A8000000E1426040E152214C0DEFF15C0DDFF43
:103A9000840E146EDECFE9FFDDCFEAFF1450EF1283
:103AA000020EE15C02E2E16AE552E16EE552E7CF27
:103AB000D9FF1200D9CFE6FFE1CFD9FF020EE126F0
:103AC000FD0EDB500FE0FE0EEA6ADB34FE0BEA3639
:103AD000E96E6D0EE926000EEA22EECFDEFFEDCF95
:103AE000DDFF0ED0FE0EEA6ADB34FE0BEA36E96E2D
:103AF000670EE926000EEA22EECFDEFFEDCFDDFFF6
:103B0000D9CFE9FFDACFEAFFEE50ED1003E1F36A17
:103B1000F46A49D0DECFE9FFDDCFEAFF020EE926E5
:103B2000000EEA22FB0EDBCFEEFFFC0EDBCFEDFF3B
:103B3000DECFE9FFDDCFEAFFEE52FA0EDBCFEFFF7B
:103B4000400E146EDECFE9FFDDCFEAFF1450EF1612
:103B5000880E146EDECFE9FFDDCFEAFF1450EF12BE
:103B6000FD0EDB500CE0FE0EEA6ADB34FE0BEA369B
:103B7000E96E6D0EE926000EEA22EF740BD0FE0E00
:103B8000EA6ADB34FE0BEA36E96E670EE926000EC0
:103B9000EA22EF74DECF14F0DDCF15F014C0F3FF8E
:103BA00015C0F4FF00D0020EE15C02E2E16AE552CA
:103BB000E16EE552E7CFD9FF1200D9CFE6FFE1CFA2
:103BC000D9FF6DA84ED0FE0EEA6ADB34FE0BEA3652
:103BD000E96E6D0EE926000EEA22EE50EFCFEAFF05
:103BE000E96E400EEE16EE6AEE6AEE6AFE0EEA6AC4
:103BF000DB34FE0BEA36E96E6D0EE926000EEA2292
:103C0000EE50EFCFEAFFE96EEE7CFE0EEA6ADB349F
:103C1000FE0BEA36E96E6D0EE926000EEA22EF741D
:103C2000400E146EFE0EEA6ADB34FE0BEA36E96ED5
:103C30006D0EE926000EEA22EE50EFCFEAFFE96EA4
:103C40001450EF16FE0EEA6ADB34FE0BEA36E96E1C
:103C50006D0EE926000EEA22EE50EFCFEAFFE96E84
:0A3C6000EF7CE552E7CFD9FF120018
:063C6A009EAC96D09E9C6A
:103C7000C3CF9FF0C4CFA0F00201FC5102E084EC5E
:103C800024F00201EAB525D09FC0E6FFA0C0E6FF00
:103C900098EC26F0E552E5520201300E7F6F806FFE
:103CA0000001DA250201816F300E0001D9250201E1
:103CB000826F300E0001D8250201836F300E0001A3
:103CC000D7250201846F3E0E856F0001030E966FAB
:103CD00064D00001A129EA6AED0FE96E020EEA2222
:103CE000EF50290803E0050EA15D32E3A1C094F076
:103CF000060E9403F3500201F8250001956F95C05C
:103D0000E6FF9451EA6AED0FE96E020EEA22EF50E7
:103D1000E66E9FC0E6FFA0C0E6FF49EC09F0E55261
:103D2000E552E552E552050E00019525EA6A7F0F3E
:103D3000E96E020EEA223E0EEF6EE66ACCEC08F067
:103D4000E5520001A16B030E966F0201EB9125D0A5
:103D5000A12BA1C0E6FFCCEC08F0E552C282000125
:103D6000A105946F060E9403F3500201F82500019B
:103D7000956F95C0E6FF9451EA6AED0FE96E020E69
:103D8000EA22EF50E66E9FC0E6FFA0C0E6FF49ECD6
:103D900009F0E552E552E552E5521200D9CFE6FFAF
:103DA000E1CFD9FF070EE126DF6A010EDB6A020EC2
:103DB000DB6A0201ECA11AD0050EDB6A060EDB6A93
:103DC000050EDB2A060E01E3DB2A000ED65C0EE3AD
:103DD000FF0ED75C0BE1050EDBCF14F0060EDBCF38
:103DE00015F0E80E145C030E1558EAE3F2A4ACD00B
:103DF000F294030ED6CFDBFF040ED7CFDBFFDBCF71
:103E000016F016C017F0166A030EDB5000011610EC
:103E1000146E17C015F0010E14C0DBFF020E15C0A2
:103E2000DBFFD950010FE96EDACFEAFF0001B05194
:103E3000EE26B151ED22010EDBCF14F0020EDBCFE6
:103E400015F015C014F0156A1450D76E010EDB5032
:103E5000D66E0201ECA178D08A7A0201540EBC6FB2
:103E6000BD6F300EBE6F720EBF6F0201ECA30FD09C
:103E7000010EDF6EEB810201F86B00019A6BC36AE1
:103E8000C46AE66ACCEC08F0E5529E9CC28202014C
:103E9000ECA52CD0E66A410EE66E8050E66E61EC31
:103EA0000CF0E552E552E552060EE66E420EE66E65
:103EB0008150E66E61EC0CF0E552E552E5520C0ED5
:103EC000E66E430EE66E8250E66E61EC0CF0E55253
:103ED000E552E5520201120EF86FDF5007E1F86B70
:103EE00002013E0E906F0001030E966F0001A65175
:103EF000A71118E00201ECB705D00001A607000EDB
:103F0000A75B0FD00001AA51AB1104E0AA07000E75
:103F1000AB5B07D0E80EAA6F030EAB6FA607000ECF
:103F2000A75B07D0A651A71104E10201EC91EB9128
:103F30008A9A0201EB51040B07E00001A55104E14C
:103F4000040EA56F976B986B070EE15C02E2E16AC5
:103F5000E552E16EE552E7CFD9FF12000201EA9582
:103F6000EA91EA93410E0201BD5D03E0420EBD5DA0
:103F70001EE1630EBF5D09E1BEC2E6FFBDC2E6FF02
:103F800091EC08F0E552E55211D0720EBF5D0EE1E2
:103F90000001630E966F976B986BBEC2E6FFBDC2C1
:103FA000E6FF91EC08F0E552E552C2824CD0430E98
:103FB000BD5D2EE14D0EBE5D2BE1650EBF5D0FE1D7
:103FC0003A0EC05D0CE10201EA85EC830001A16BB1
:103FD00001EC09F0E66ACCEC08F0E55218D0640E6A
:103FE000BF5D03E10201EC9312D0720EBF5D0FE1E1
:103FF0000201EA850201F86B0001A16B630E966F66
:10400000976B986BE66ACCEC08F0E552C2821BD045
:10401000560EBD5D12E1500EBE5D0FE1650EBF5D37
:1040200005E1C1880001010EA46F06D0640EBF5DDA
:1040300003E1C1980001A46B06D0540EBD5D03E1FD
:10404000560EBE5D00E1120012001200500E020179
:10405000BD5D32E1770EBF5D26E10001946B080E75
:10406000945D20E2060E9425EA6ABB0FE96E020E0B
:10407000EA22EF50780813E0060E9425EA6ABB0F97
:10408000E96E020EEA22EF50E66E300E9425E66EDF
:10409000BEC2E6FF71EC0AF0E552E552E5520001BE
:1040A000942BDDD708D0720EBF5D05E1BEC2E6FFDE
:1040B000E7EC09F0E552BCD0430EBD5D3BE14D0E8F
:1040C000BE5D38E1650EBF5D03E10201EC8531D0D4
:1040D000640EBF5D03E10201EC952BD0720EBF5D53
:1040E00028E1E66A410EE66E8050E66E61EC0CF067
:1040F000E552E552E552060EE66E420EE66E81503E
:10410000E66E61EC0CF0E552E552E5520C0EE66EFF
:10411000430EE66E8250E66E61EC0CF0E552E5521D
:10412000E55202013E0E906F0201F86B0001030E92
:10413000966F7ED0550EBD5D10E1420EBE5D05E16D
:10414000650EBF5D02E1F19E07D0420EBE5D04E147
:10415000640EBF5D01E1F18E6BD04D0EBD5D68E177
:10416000650EBF5D03E0640EBF5D09E1BFC2E6FFFF
:10417000BEC2E6FFE3EC0CF0E552E55259D0660E04
:10418000BF5D1FE16B0EC45D1CE1C3C2E6FFC2C28E
:10419000E6FFC1C2E6FF300EE66EE66EF9EC25F0F2
:1041A000146E050EE15E1450F3CF9DF0F4CF9EF037
:1041B0009DC0E6FF9EC0E6FF70EC0DF0E552E552B3
:1041C00037D0720EBF5D34E1C4C2E6FFC3C2E6FF62
:1041D000C2C2E6FFC1C2E6FF300EE66EF9EC25F082
:1041E000146E050EE15E1450F3CF9DF0F4CF9EF0F7
:1041F0000001000ED8809D55000E9E5503E29D2BB8
:10420000000E9E239DC014F09EC015F0166A176A1A
:1042100014C0E6FF15C0E6FF16C0E6FF17C0E6FFB4
:10422000BEC2E6FF10EC0DF0186E050EE15E1850F0
:104230001200BFC2E6FFBEC2E6FFBDC2E6FF71ECE0
:104240000AF0E552E552E5521200300E0201BE5D61
:1042500001E0B2D0700EBF5D06E1C1C2E6FF1DEC09
:104260000EF0E552A8D0640EBF5D09E10201EC91A9
:10427000300EE66E1DEC0EF0E5528A9A9CD0710E5F
:10428000BF5D34E1C5C2E6FFC4C2E6FFC3C2E6FFBC
:10429000C2C2E6FFC1C2E6FFF9EC25F0146E050EBE
:1042A000E15E1450F3CF9DF0F4CF9EF0176A186AC8
:1042B000010E196E9DC01AF09EC01BF01C6A1A50A8
:1042C000175C146E1B501858156E1C501958166E3A
:1042D00014C0B0F015C0B1F0F294B0C0E6FFB1C0A8
:1042E000E6FF85EC32F0E552E55265D0740EBF5D15
:1042F00031E1C3C2E6FFC2C2E6FFC1C2E6FF300E33
:10430000E66EE66EF9EC25F0146E050EE15E1450D3
:10431000F3CF9DF0F4CF9EF0C4C2E6FF9DC0E6FF50
:104320009EC0E6FF6DEC0EF0E552E552E552F3CF8C
:10433000B0F0F4CFB1F000010A0ED8809D55000E08
:104340009E5505E30201EB850001A56B02D0020139
:10435000EB9531D0630EBF5D25E1C4C2E6FFC3C259
:10436000E6FFC2C2E6FFC1C2E6FF300EE66EF9EC20
:1043700025F0146E050EE15E1450F3CF9DF0F4CFDE
:104380009EF000019D519E110CE09DC0A8F09EC0C2
:10439000A9F0010EA85F000EA95BA8C0A6F0A9C0F5
:1043A000A7F009D0720EBF5D06E10201EC81A8C042
:1043B000A6F0A9C0A7F071D0310EBE5D6EE1700EFF
:1043C000BF5D06E1C1C2E6FFEFEC10F0E55265D03B
:1043D000640EBF5D06E1300EE66EEFEC10F0E552C4
:1043E0005CD0720EBF5D34E1C5C2E6FFC4C2E6FF19
:1043F000C3C2E6FFC2C2E6FFC1C2E6FFF9EC25F088
:10440000146E050EE15E1450F3CF9DF0F4CF9EF0D4
:10441000176A186A010E196E9DC01AF09EC01BF033
:104420001C6A1A50175C146E1B501858156E1C50DD
:104430001958166E14C0B2F015C0B3F09E90B2C0F9
:10444000E6FFB3C0E6FF69EC32F0E552E55225D055
:10445000740EBF5D22E1C3C2E6FFC2C2E6FFC1C265
:10446000E6FF300EE66EE66EF9EC25F0146E050EF2
:10447000E15E1450F3CF9DF0F4CF9EF0C4C2E6FF8E
:104480009DC0E6FF9EC0E6FF1FEC11F0E552E5522D
:10449000E552F3CFB2F0F4CFB3F012004D0E0201AB
:1044A000BD5D1DE1440EBE5D1AE1720EBF5D17E1F8
:1044B000310EE66E300EE66E760EE66E320EE66E6B
:1044C000310EE66E500EE66E430EE66E690EE66E37
:1044D000D3EC25F0146E080EE15E145085D0460E24
:1044E000BD5D1CE1570EBE5D19E1720EBF5D16E1A8
:1044F000300EE66E340EE66E310EE66E300EE66E6F
:10450000E66E320EE66E310EE66E300EE66ED3ECDF
:1045100025F0146E080EE15E145066D0490EBD5DA4
:104520001BE1440EBE5D18E1720EBF5D15E199DA24
:10453000F4C2E6FFF5C2E6FFF6C2E6FFF7C2E6FF09
:10454000300EE66EE66EE66EE66ED3EC25F0146E87
:10455000080EE15E145048D0440EBD5D10E1300EEF
:10456000BF5D146E300EBE5D0A0DF35014240201BF
:10457000FC6F00019B6B9C6B010E966F35D0530E48
:10458000BD5D14E1490EBE5D11E1770EBF5D0EE128
:104590009268CF0E936E94680F0EC16E806A816A26
:1045A000826A0001966B0201FB6B1ED0520EBD5D4C
:1045B0001BE14F0EBE5D18E1520EBF5D15E1C4C296
:1045C000E6FFC3C2E6FFC2C2E6FFC1C2E6FFD1EC0E
:1045D00029F0E552E552E552E552F3CF9FF0F4CFD2
:1045E000A0F00001010E966F12000001966BA36B04
:1045F0000201FB6B0201FC6B0201EC91EC93EC9568
:10460000EA91EA93EA95EB91EB950001A56B120014
:104610000201D151EA6A3F0FE96E020EEA22EF5021
:10462000280854E10201F96BA5D90201D151EA6AC7
:104630003F0FE96E020EEA22EF50E66E0201F951D9
:10464000EA6ABB0FE96E020EEA22E552E750EF6E0E
:104650000201D151EA6A3F0FE96E020EEA22EF6AC7
:104660000201F92B0201D12B0201D0510201D15DCF
:104670000DE2D151EA6A3F0FE96E020EEA22EF50D5
:10468000290804E0140E0201F95DCEE373D902019A
:10469000D151EA6A3F0FE96E020EEA22EF50E66E50
:1046A0000201F951EA6ABB0FE96E020EEA22E552F5
:1046B000E750EF6EF951EA6ABB0FE96E020EEA228B
:1046C000EF50290803E10201010EFB6F1200020105
:1046D000FB052EE1000196512BE10201BC515A0A63
:1046E00019E00E0A15E0060A11E0020A0DE0160AAA
:1046F00009E0020A05E0050A01E00ED02FDC0CD02B
:10470000A3DC0AD0A2DC08D0A1DC06D092DD04D064
:104710009CDD02D0C3DE00D00001965102E1F3EC33
:1047200012F00001965102E1010E966F0201BB6B7F
:1047300012000001965102E1E6D070D096050EE11C
:10474000966B0201CF51EA6A000FE96E010EEA2270
:10475000230EEF6ECF2B0201FB6B60D0020E965D35
:1047600003E0030E965D5AE1A55101E0A507020E94
:10477000965D03E1080E956F05D0030E965D02E18C
:104780003C0E956F966BBFC2E6FFBEC2E6FFBDC290
:10479000E6FFBCC2E6FF22EC08F0E552E552E55226
:1047A000E5520001946B942B9451EA6A7F0FE96EF5
:1047B000020EEA22EF503E0803E09551945DF3E3C8
:1047C0009451E66EE66A7F0EE66E020EE66E020118
:1047D000CF51156A000F146E010E152214C0E6FFAA
:1047E00015C0E6FF0DEC31F0166E060EE15E1650B8
:1047F00000019451EA6A7F0FE96E020EEA22EF6A25
:1048000094510201CF27CF51EA6A000FE96E010EE1
:10481000EA223E0EEF6ECF2B0201FB6B630E00010E
:10482000965D07E00201EB51010B03E10001A55188
:104830000DE00001972B000E9823280E975D230EA4
:10484000985904E3976B986BCD0E966F9651146E42
:10485000156A153404E21450C808000E155453E2CA
:1048600096519F6FA06BC80E9F5F000EA05B9FC00C
:10487000E6FFA0C0E6FF98EC26F0E552E552020103
:10488000CF51EA6A000FE96E010EEA223C0EEF6E8C
:10489000CF29EA6A000FE96E010EEA225A0EEF6E86
:1048A000020ECF25EA6A000FE96E010EEA22450EDC
:1048B000EF6E300E0001D825E66E030E0201CF2503
:1048C000EA6A000FE96E010EEA22E552E750EF6E48
:1048D000300E0001D725E66E040E0201CF25EA6AEC
:1048E000000FE96E010EEA22E552E750EF6E050E69
:1048F000CF25EA6A000FE96E010EEA223E0EEF6E46
:10490000060ECF2772DE12000201FC0511E1000144
:10491000E80E9B5D030E9C5903E39B6B9C6B03D0DD
:104920009B2B000E9C239BC09FF09CC0A0F021D02D
:10493000020EFC5D07E12DEC32F0F3CF9FF0F4CFD7
:10494000A0F017D0030EFC5D11E100019A2B300E90
:104950009A25E66E0201CF51EA6A000FE96E010E58
:10496000EA22E552E750EF6ECF2B03D0040EFC5D38
:1049700000E112000B0E0201FC5D0EE1ACA2FED7BD
:104980000201D151EA6A3F0FE96E020EEA22EF50AE
:10499000E66E57EC2BF0E5521200D9CFE6FFE1CFDF
:1049A000D9FF040EE12600019F6BA06BFF0EE66E9F
:1049B000010EE66E9FC014F0A0C015F0166A176ACB
:1049C00014C0E6FF15C0E6FF16C0E6FF17C0E6FFFD
:1049D00011EC14F0186E060EE15E1850FFC1DFFFF7
:1049E000010E00C2DBFF0001200E9F6F080EA06FBA
:1049F000FF0EE66E010EE66E9FC014F0A0C015F02B
:104A0000166A176A14C0E6FF15C0E6FF16C0E6FF77
:104A100017C0E6FF11EC14F0186E060EE15E185098
:104A2000020EFFC1DBFF030E00C2DBFFDF500DE112
:104A3000010EDB500AE1020EDB50ED0806E1030E29
:104A4000DB50100802E103D002D08A8AFFD7040E9F
:104A5000E15C02E2E16AE552E16EE552E7CFD9FF9F
:104A60001200D9CFE6FFE1CFD9FF040EE1263F0EB9
:104A7000F86EF768FE0EF66E0800F550DF6EF66809
:104A80000800010EF5CFDBFF0F0EDF14E76E020EFC
:104A9000E7CFDBFFDF380F0B0F0BE76E030EE7CF1F
:104AA000DBFF020EDB50090806E2020EDB50370F77
:104AB0000201F46F05D0020EDB50300F0201F46FDB
:104AC000030EDB50090806E2030EDB50370F02012C
:104AD000F56F05D0030EDB50300F0201F56F010EAC
:104AE000DB500F0BE76E020EE7CFDBFF010EDB386A
:104AF0000F0B0F0BE76E030EE7CFDBFF020EDB5051
:104B0000090806E2020EDB50370F0201F66F05D0EE
:104B1000020EDB50300F0201F66F030EDB50090866
:104B200006E2030EDB50370F0201F76F05D0030ECC
:104B3000DB50300F0201F76F040EE15C02E2E16A24
:0C4B4000E552E16EE552E7CFD9FF12000C
:044B4C00D9CFE6FFD8
:104B5000E1CFD9FFFD0EDBCFE9FFFE0EDBCFEAFF91
:104B6000EF501DE0FD0EDBCFE9FFFE0EDBCFEAFFCD
:104B7000EF50E66E0201CF51EA6A000FE96E010EB6
:104B8000EA22E552E750EF6ECF2BFD0EDBCFE9FFB7
:104B9000DB2AFE0EDBCFEAFF01E3DB2ADBD7E5529F
:104BA000E7CFD9FF1200D9CFE6FFE1CFD9FFFE0E44
:104BB000DBCF7FF2FD0EDBCF80F2FC0EDBCF81F28C
:104BC000FB0EDBCF82F2FA0EDBCF83F2F90EDBCFE6
:104BD00084F2F80EDBCF85F2F70EDBCF86F202010E
:104BE0003E0E876F0001020E966FE552E7CFD9FFA8
:104BF0001200D9CFE6FFE1CFD9FF020EE126DE6A2F
:104C0000DD6AFE0EDBCF14F0156A14BE1568300E97
:104C1000145E000E155A100E1502F3CF15F0270E74
:104C20001402F3501526100E1402F3CF14F0F450B2
:104C3000152614C0DEFF15C0DDFFFD0EDBCF14F01E
:104C4000156A14BE1568300E145E000E155AE80E73
:104C50001502F3CF15F0030E1402F3501526E80EDB
:104C60001402F3CF14F0F4501526D9CFE9FFDACFB0
:104C7000EAFF1450EE261550ED22FC0EDBCF14F0A7
:104C8000156A14BE1568300E145E000E155A640EB7
:104C90001502F3CF15F01402F3CF14F0F4501526DB
:104CA000D9CFE9FFDACFEAFF1450EE261550ED22F6
:104CB000FB0EDBCF14F0156A14BE1568300E145EBF
:104CC000000E155A0A0E1502F3CF15F01402F3CF99
:104CD00014F0F4501526D9CFE9FFDACFEAFF1450CB
:104CE000EE261550ED22FA0EDBCF14F0156A14BE35
:104CF0001568300E145E000E155AD9CFE9FFDACFD1
:104D0000EAFF1450EE261550ED22DECF14F0DDCF71
:104D100015F014C0F3FF15C0F4FF020EE15C03E2CE
:104D200000D0E16AE552E16EE552E7CFD9FF12000B
:104D3000D9CFE6FFE1CFD9FF0001DB6BDA6BD96B8E
:104D4000D86BD76BD950FD0FE96EFF0EDA20EA6EF3
:104D5000EE50ED1001E121D3FD0EDBCF14F0FE0E7D
:104D6000DBCF15F0D890155004E6E80E145C030E66
:104D7000155801E283D0FD0EDBCF14F0FE0EDBCF21
:104D800015F0D890155004E6A00E145C0F0E1558BF
:104D900013E3040EDA6FFD0EDBCF14F0FE0EDBCF53
:104DA00015F0A00E145E0F0E155AFD0E14C0DBFF99
:104DB000FE0E15C0DBFF62D0FD0EDBCF14F0FE0E41
:104DC000DBCF15F0D890155004E6B80E145C0B0E2E
:104DD000155813E3030EDA6FFD0EDBCF14F0FE0E51
:104DE000DBCF15F0B80E145E0B0E155AFD0E14C075
:104DF000DBFFFE0E15C0DBFF41D0FD0EDBCF14F054
:104E0000FE0EDBCF15F0D890155004E6D00E145CE2
:104E1000070E155813E3020EDA6FFD0EDBCF14F008
:104E2000FE0EDBCF15F0D00E145E070E155AFD0EE8
:104E300014C0DBFFFE0E15C0DBFF20D0FD0EDBCF64
:104E400014F0FE0EDBCF15F0D890155004E6E80EF6
:104E5000145C030E155812E3010EDA6FFD0EDBCF62
:104E600014F0FE0EDBCF15F0E80E145E030E155A9B
:104E7000FD0E14C0DBFFFE0E15C0DBFFFD0EDBCF09
:104E800014F0FE0EDBCF15F0D890155004E6F40EAA
:104E9000145C010E155801E2A5D0FD0EDBCF14F015
:104EA000FE0EDBCF15F0D890155004E6840E145C8E
:104EB000030E155813E3090ED96FFD0EDBCF14F066
:104EC000FE0EDBCF15F0840E145E030E155AFD0E98
:104ED00014C0DBFFFE0E15C0DBFF83D0FD0EDBCF61
:104EE00014F0FE0EDBCF15F0D890155004E6200E1E
:104EF000145C030E155813E3080ED96FFD0EDBCFBB
:104F000014F0FE0EDBCF15F0200E145E030E155AC2
:104F1000FD0E14C0DBFFFE0E15C0DBFF62D0FD0EE0
:104F2000DBCF14F0FE0EDBCF15F0D890155004E661
:104F3000BC0E145C020E155813E3070ED96FFD0E5C
:104F4000DBCF14F0FE0EDBCF15F0BC0E145E020EAC
:104F5000155AFD0E14C0DBFFFE0E15C0DBFF41D05D
:104F6000FD0EDBCF14F0FE0EDBCF15F0D890155000
:104F700004E6580E145C020E155813E3060ED96FA2
:104F8000FD0EDBCF14F0FE0EDBCF15F0580E145ED5
:104F9000020E155AFD0E14C0DBFFFE0E15C0DBFF1E
:104FA00020D0FD0EDBCF14F0FE0EDBCF15F0D89035
:104FB000155004E6F40E145C010E155812E3050EAC
:104FC000D96FFD0EDBCF14F0FE0EDBCF15F0F40E23
:104FD000145E010E155AFD0E14C0DBFFFE0E15C047
:104FE000DBFF92D0FD0EDBCF14F0FE0EDBCF15F011
:104FF000D890155004E6640E145C000E155801E2BA
:1050000083D0FD0EDBCF14F0FE0EDBCF15F0D89071
:10501000155004E6900E145C010E155813E3040EAF
:10502000D96FFD0EDBCF14F0FE0EDBCF15F0900E26
:10503000145E010E155AFD0E14C0DBFFFE0E15C0E6
:10504000DBFF62D0FD0EDBCF14F0FE0EDBCF15F0E0
:10505000D890155004E62C0E145C010E155813E37D
:10506000030ED96FFD0EDBCF14F0FE0EDBCF15F073
:105070002C0E145E010E155AFD0E14C0DBFFFE0E41
:1050800015C0DBFF41D0FD0EDBCF14F0FE0EDBCFF1
:1050900015F0D890155004E6C80E145C000E155893
:1050A00013E3020ED96FFD0EDBCF14F0FE0EDBCF43
:1050B00015F0C80E145E000E155AFD0E14C0DBFF6D
:1050C000FE0E15C0DBFF20D0FD0EDBCF14F0FE0E70
:1050D000DBCF15F0D890155004E6640E145C000E7A
:1050E000155812E3010ED96FFD0EDBCF14F0FE0E42
:1050F000DBCF15F0640E145E000E155AFD0E14C0C1
:10510000DBFFFE0E15C0DBFFFD0EDBCF14F0FE0E45
:10511000DBCF15F0D890155004E6320E145C000E6B
:10512000155801E2A5D0FD0EDBCF14F0FE0EDBCF4B
:1051300015F0D890155004E65A0E145C000E155860
:1051400013E3090ED86FFD0EDBCF14F0FE0EDBCF9C
:1051500015F05A0E145E000E155AFD0E14C0DBFF3A
:10516000FE0E15C0DBFF83D0FD0EDBCF14F0FE0E6C
:10517000DBCF15F0D890155004E6500E145C000EED
:10518000155813E3080ED86FFD0EDBCF14F0FE0E9A
:10519000DBCF15F0500E145E000E155AFD0E14C034
:1051A000DBFFFE0E15C0DBFF62D0FD0EDBCF14F07F
:1051B000FE0EDBCF15F0D890155004E6460E145CB9
:1051C000000E155813E3070ED86FFD0EDBCF14F059
:1051D000FE0EDBCF15F0460E145E000E155AFD0EC6
:1051E00014C0DBFFFE0E15C0DBFF41D0FD0EDBCF90
:1051F00014F0FE0EDBCF15F0D890155004E63C0EEF
:10520000145C000E155813E3060ED86FFD0EDBCFAD
:1052100014F0FE0EDBCF15F03C0E145E000E155A96
:10522000FD0E14C0DBFFFE0E15C0DBFF20D0FD0E0F
:10523000DBCF14F0FE0EDBCF15F0D890155004E64E
:10524000320E145C000E155812E3050ED86FFD0ED9
:10525000DBCF14F0FE0EDBCF15F0320E145E000E25
:10526000155AFD0E14C0DBFFFE0E15C0DBFF92D0F9
:10527000FD0EDBCF14F0FE0EDBCF15F0D8901550ED
:1052800004E60A0E145C000E155801E283D0FD0EF0
:10529000DBCF14F0FE0EDBCF15F0D890155004E6EE
:1052A000280E145C000E155813E3040ED86FFD0E83
:1052B000DBCF14F0FE0EDBCF15F0280E145E000ECF
:1052C000155AFD0E14C0DBFFFE0E15C0DBFF62D0C9
:1052D000FD0EDBCF14F0FE0EDBCF15F0D89015508D
:1052E00004E61E0E145C000E155813E3030ED86F6F
:1052F000FD0EDBCF14F0FE0EDBCF15F01E0E145E9C
:10530000000E155AFD0E14C0DBFFFE0E15C0DBFFAC
:1053100041D0FD0EDBCF14F0FE0EDBCF15F0D890A0
:10532000155004E6140E145C000E155813E3020E1B
:10533000D86FFD0EDBCF14F0FE0EDBCF15F0140E90
:10534000145E000E155AFD0E14C0DBFFFE0E15C0D4
:10535000DBFF20D0FD0EDBCF14F0FE0EDBCF15F00F
:10536000D890155004E60A0E145C000E155812E38E
:10537000010ED86FFD0EDBCF14F0FE0EDBCF15F063
:105380000A0E145E000E155AFD0E14C0DBFFFE0E51
:1053900015C0DBFFFD0EDBCFD7F0E552E7CFD9FF1D
:1053A0001200D9CFE6FFE1CFD9FF0A0EE126FE0EAB
:1053B000DB5039080EE3FE0EDB50D00F146E156A79
:1053C00014BE1568080E14C0DBFF090E15C0DBFF04
:1053D00011D0FE0EDB5039080DE2FE0EDB50C90F76
:1053E000146E156A14BE1568080E14C0DBFF090E92
:1053F00015C0DBFF086A100E096E080EDBCF0DF03A
:10540000090EDBCF0EF03BEC30F0080E06C0DBFFE0
:10541000090E07C0DBFFFD0EDB5039080EE3FD0E61
:10542000DB50D00F146E156A14BE1568060E14C03A
:10543000DBFF070E15C0DBFF11D0FD0EDB50390876
:105440000DE2FD0EDB50C90F146E156A14BE15680F
:10545000060E14C0DBFF070E15C0DBFF086A010E45
:10546000096E060EDBCF0DF0070EDBCF0EF03BEC26
:1054700030F0060E06C0DBFF070E07C0DBFFFC0E98
:10548000DB5039080EE3FC0EDB50D00F146E156AAA
:1054900014BE1568040E14C0DBFF050E15C0DBFF3B
:1054A00011D0FC0EDB5039080DE2FC0EDB50C90FA9
:1054B000146E156A14BE1568040E14C0DBFF050EC9
:1054C00015C0DBFF100E086E096A040EDBCF0DF06D
:1054D000050EDBCF0EF03BEC30F0040E06C0DBFF18
:1054E000050E07C0DBFFFB0EDB5039080EE3FB0E99
:1054F000DB50D00F146E156A14BE1568020E14C06E
:10550000DBFF030E15C0DBFF11D0FB0EDB503908AB
:105510000DE2FB0EDB50C90F146E156A14BE156840
:10552000020E14C0DBFF030E15C0DBFF060EDBCF3F
:105530001AF0070EDBCF1BF0080EDB501A24186E92
:10554000090EDB501B20196E040EDB501824166E5A
:10555000050EDB501920176E020EDB501624146E58
:10556000030EDB501720156E14C0DEFF15C0DDFFE3
:10557000DECF14F0DDCF15F014C0F3FF15C0F4FF3B
:105580000A0EE15C03E200D0E16AE552E16EE55209
:06559000E7CFD9FF120075
:0A559600DACFE4FFE2CFDAFFE652BD
:1055A000E552E5CFDAFF1100D8CFE4FFE0CFE4FF0A
:1055B000E46EDACFE4FFE2CFDAFFE652E552E5CF60
:1055C000DAFFE550E5CFE0FFE5CFD8FF100011D8B6
:1055D0000201EBB102D070EC15F00201EBB105D085
:1055E00005D967EC23F0CEEC1EF035EC1EF0F0D7B9
:1055F00012000F0EC11202D8E4EF14F0D9CFE6FF6B
:10560000E1CFD9FFE652DF6ADF50146E156AFF0E54
:10561000145C000E155809E2DF50EA6A000FE96ECB
:10562000010EEA22EF6ADF2AEFD70201CF6BD06BBF
:10563000D26BD36BCF0E93169268936E9468C26A46
:105640000F0EC16EBE0EC06E070EB46E806A816A08
:10565000826ADF6A080EDF5C09E2DF50EA6A7F0FC8
:10566000E96E020EEA22EF6ADF2AF4D7F5EC22F0A7
:10567000CDEC24F0E552E552E7CFD9FF1200D9CFA7
:10568000E6FFE1CFD9FFE652938A939E240EAC6EDB
:10569000900EAB6E710EAF6E020EB06E080EB86E4D
:1056A000AE50DF6EE552E552E7CFD9FF1200D9CFF9
:1056B000E6FFE1CFD9FFFE0EDB50AD6EE552E7CF3E
:1056C000D9FF1200D9CFE6FFE1CFD9FF050EE126C1
:1056D000A00E0501001907E1860E011904E1010E73
:1056E000021901E1035116E10201010EFA6F9396CE
:1056F00081966D926D6ADF6AFF0EDF5C09E2E868F1
:10570000E85004E0E80600D000D0FAD7DF2AF4D74A
:1057100000EF00F0D880000E05010055C20E0155C3
:10572000010E0255000E035501E241D000C5CFF530
:1057300001C5D0F502C5D1F503C5D2F5186A1B0E17
:10574000196EB70E1A6E1B6A18C006F019C007F062
:105750001AC008F01BC009F0CFC50BF0D0C50CF083
:10576000D1C50DF0D2C50EF0E8EC31F006C014F052
:1057700007C015F008C016F009C017F01406000E97
:10578000155A000E165A000E175A010E14C0DBFFF0
:10579000020E15C0DBFF030E16C0DBFF040E17C0A0
:1057A000DBFF010EDB50AF6E020EDB50B06E050E5C
:1057B000E15C02E2E16AE552E16EE552E7CFD9FF32
:1057C0001200D9CFE6FFE1CFD9FFE652ABA205D058
:1057D000AB98AE50DF6EAB8802D0AE50DF6EDF50BC
:1057E00000D0E552E552E7CFD9FF1200D9CFE6FF4E
:1057F000E1CFD9FFE6520A0E0201FC5D03E10B0E78
:10580000FC6F3DDF200E0001E76E6019E8AE02D0AC
:10581000E73402D0E750605D03E36D50020B01E016
:10582000B4D00201FD5115E1400EE66E3F0EE66E6A
:10583000020EE66E11EC2EF0E552E552E552020141
:10584000D06FD051000805E20201010EFD6F020188
:10585000D16B0201FD5111E0AC50020B0EE0FB5187
:105860000CE10001965109E108EC23F00201D12B73
:10587000D051D15D02E30201FD6B0001B55102E19F
:1058800099EC23F00B0E0201FC5D50E19E50200BC1
:105890004DE00201CF51146E156AD890155004E600
:1058A000860E145C000E155841E28BDFE66E020195
:1058B000CF51EA6A000FE96E010EEA22E552E75085
:1058C000EF6ECF51EA6A000FE96E010EEA22EF5047
:1058D000280802E10201F96B0201CF51EA6A000FC8
:1058E000E96E010EEA22EF50290803E10201010EE0
:1058F000FB6F0201CF51EA6A000FE96E010EEA2246
:10590000EF50E66E0201F951EA6ABB0FE96E020E32
:10591000EA22E552E750EF6EF92B0201CF2BCF516F
:10592000EA6A000FE96E010EEA22EF6A0001B55142
:105930002AE10201CF51000826E20001A55123E12E
:10594000CFC2E6FF000EE66E010EE66E72EC2EF0A0
:10595000E552E552E5520B0E0201FC5D12E1DF6AF1
:10596000ACA2FED7DF50EA6A000FE96E010EEA2210
:10597000EF50E66E9CDEE552DF2A0201CF51DF5C7C
:10598000EFE30201CF6B0EEC2FF0E552E552E7CFCB
:10599000D9FF12000201FE51FF1104E1100EFE6F4B
:1059A000270EFF6FFE07000EFF5B6DA20AD0FE51AF
:1059B000FF1106E18A788AA802D08A8A01D08A9AE1
:1059C0002ED00001605103E18A988A9A28D06005A0
:1059D00003E18A888A8A23D0020E605D03E18A8807
:1059E0008A9A1DD0040E605D03E18A988A8A17D0D6
:1059F000100E605D07E10201FE51FF1102E18A789D
:105A00008A9A0DD0200E605D0AE10201FE51FF115D
:105A100006E18A788AA802D08A9A01D08A8A12007E
:105A200012001200120012008AEF2DF01200DDEFBA
:105A30002DF0000183051EE1000184051BE1F1DF6B
:105A40006D920001846B0201100ED46F0E0ED56FA3
:105A5000D407000ED55BD451D511FAE16D84080E40
:105A6000D46F070ED56FD407000ED55BD451D51176
:105A7000FAE16D941200D9CFE6FFE1CFD9FFFD0E18
:105A8000DBCF08F0FE0EDBCF09F0050E081801E1B0
:105A9000095039E0E868081802E17F0E091831E082
:105AA000030E081801E109502AE0020E081801E16E
:105AB000095023E0010E081801E109501CE0740EA2
:105AC000081801E1095015E0750E081801E10950A8
:105AD0000EE0730E081801E1095007E0720E081875
:105AE00001E1095001E010D00FD09CDF0DD098DF0C
:105AF0000BD097DF09D09BDF07D098DF05D094DF6C
:105B000003D091DF01D000D0010E00D0E552E7CFE5
:045B1000D9FF1200A7
:0C5B1400040130511F0B010801E04CD0CF
:105B20003051600BE842E842E842E842E8420108AE
:105B300001E042D0345103E0340501E03DD0315161
:105B4000220A35E0030A28E0010A17E0210A0EE0E4
:105B5000010A01E031D00001C50E756F000E766FAD
:105B6000080E786F796B7781778F26D00001C50E8C
:105B7000756F000E766F778F1FD036C47DF037C4F7
:105B80007EF00001000E7A6F050E7B6FC40E7F6FF2
:105B9000560E806F7C8F10D00001CF0E756F050EF2
:105BA000766F070E786F796BC10E776F05D032C4B0
:105BB000C0F00001778F00D012000501CF6B4B0EB3
:105BC000D06FD16BD26BD36BD46B080ED56F000145
:105BD000B46B1A0EE66E010EE66EB3EC1CF0E552E5
:105BE000E5521E0EE66E020EE66EB3EC1CF0E552B8
:105BF000E552870EE66E080EE66E050EE66EE66A64
:105C0000020EE66E5AEC1DF0146E050EE15E1450A5
:105C1000F3CFBCF0F4CFBDF00001BE6BBF6BB56B32
:105C20001200D9CFE6FFE1CFD9FF0001B46BBC5120
:105C3000BD1102E1000E08D0BCC0E9FFBDC0EAFF03
:105C4000EF50800B01E0010E000945E1FC0EDBCFB7
:105C500014F0BCC0E9FFBDC0EAFFEE52EF50D8809F
:105C6000145408E2BCC0E9FFBDC0EAFFEE52FC0ECE
:105C7000EFCFDBFFB46BFC0EDB50B45D19E2B45127
:105C8000EA6A080FE96E050EEA22EF50E66EB4519B
:105C9000E76EFD0EDBCFE9FFFE0EDBCFEAFFE7503C
:105CA000E926000EEA22E552E750EF6EB42BE3D767
:105CB000870EE66E080EE66E050EE66EE66A020ECA
:105CC000E66E5AEC1DF0146E050EE15E1450F3CF33
:105CD000BCF0F4CFBDF00001B45100D0E552E7CFE5
:105CE000D9FF1200D9CFE6FFE1CFD9FF0001B551AE
:105CF0000CE1FD0EDBCFB6F0FE0EDBCFB7F0FC0EF5
:105D0000DBCFBAF0010EBB6FB56FE552E7CFD9FF1D
:105D10001200D9CFE6FFE1CFD9FF030EE126000143
:105D2000B55101E02ED0DF6AFD0EDBCF08F0FE0E8C
:105D3000DBCF09F0DE5208C0DEFF09C0DDFFDD5217
:105D4000DF2ADF50146E156AFF0E141801E115509A
:105D500001E10BD0010EDBCFE9FFDB2A020EDBCF26
:105D6000EAFF01E3DB2AEF50EBE1FD0EDBCFB6F0FB
:105D7000FE0EDBCFB7F0DFCFBAF00001010EBB6F34
:105D8000B56F030EE15C02E2E16AE552E16EE552B5
:105D9000E7CFD9FF1200D9CFE6FFE1CFD9FF030E3D
:105DA000E1260001B55101E02FD0DF6AFD0EDBCF07
:105DB00008F0FE0EDBCF09F0DE5208C0DEFF09C09E
:105DC000DDFFDD52DF2ADF50146E156AFF0E141856
:105DD00001E1155001E10CD0010EDBCFF6FFDB2A0B
:105DE000020EDBCFF7FF01E3DB2A0800F550EAE102
:105DF000FD0EDBCFB6F0FE0EDBCFB7F0DFCFBAF093
:105E00000001BB6B010EB56F030EE15C02E2E16ABB
:105E1000E552E16EE552E7CFD9FF1200D9CFE6FF98
:105E2000E1CFD9FF020EE1260001BE51BF1102E110
:105E3000000E08D0BEC0E9FFBFC0EAFFEF50800BE4
:105E400001E0010E000901E085D0030EB55D01E11E
:105E5000B56BB55101E17ED0020EB55D16E1E66A83
:105E6000000EE66EE66A010EE66E020EE66E5AEC73
:105E70001DF0146E050EE15E1450F3CFBEF0F4CFAA
:105E8000BFF00001030EB56F65D0B50563E1400EAC
:105E9000146E156ABA51145C000E155803E2400ED8
:105EA000DF6E02D0BAC0DFFFDF50BA5DBA6F8F0E6F
:105EB000B86F050EB96F010EDFCFDBFFBB5117E1E5
:105EC000010EDB5013E0B6C0F6FFB7C0F7FF0800C5
:105ED000F550B8C0E9FFB9C0EAFFEF6EB82B000E6D
:105EE000B923B62BB723010EDB06EAD715D0010E76
:105EF000DB5012E0B6C0E9FFB7C0EAFFEF50B8C010
:105F0000E9FFB9C0EAFFEF6EB82B000EB923B62B3C
:105F1000B723010EDB06EBD7BA5108E1400EDF5C78
:105F200003E1020EB56F02D0030EB56FDFCFE6FFBF
:105F30008F0EE66E050EE66E010EE66E020EE66E42
:105F40005AEC1DF0146E050EE15E1450F3CFBEF056
:105F5000F4CFBFF0020EE15C02E2E16AE552E16ECD
:085F6000E552E7CFD9FF120062
:085F6800006A0EAEBDEF2FF040
:105F70000D6C0E1EE86A0E22001E09AEC5EF2FF052
:105F8000086C091EE86A0922001ED8EC32F009BE2E
:105F9000D5EF2FF000AE000C086C091EE86A09224C
:105FA000046C051EE86A0522000C00BECCEF2FF041
:105FB0000188FF0C006A0EAEE5EF2FF00C6C0D1E91
:105FC0000E1EE86A0D220E22001E09AEEFEF2FF022
:105FD000076C081E091EE86A08220922001E4CEC04
:105FE00032F009BE02EF30F000AE000C076C081E64
:105FF000091EE86A08220922036C041E051E0422F9
:106000000522000C00BEF6EF2FF00188FF0C006A9D
:10601000E86A0EAE14EF30F00B6C0C1E0D1E0E1E57
:106020000C220D220E22001E09AE1FEF30F0066C6E
:10603000071E081E091E072208220922001EE8EC7E
:1060400031F009BE36EF30F000AE000C066C071ED2
:10605000081E091EE86A072208220922026C031E94
:10606000041E051E032204220522000C00BE26EF9A
:1060700030F00188FF0C08C012F008500D02F4CF78
:1060800007F0F3CF06F009500E02F4CF09F0F3CF7A
:1060900008F00D02F3500726F4500822E86A09229E
:1060A00012500E02F3500726F4500822E86A092223
:0260B000000CE2
:0E60B2001201000202000008D8040A000001DA
:1060C0000102000109024300020100C0320904007C
:1060D000000102020100052400100104240202054F
:1060E00024060001052401000107058103080002C0
:1060F00009040100020A0000000705020240000036
:1061000007058202400000040309043403690043C8
:10611000006900720063007500690074002000547B
:10612000006500630068006E006F006C006F006720
:1061300000690065007300000000000000000034EA
:1061400003690043005000310032002000620079F2
:1061500000200050004900430063006900720063A2
:10616000007500690074002E0063006F006D002050
:0B617000000000C46007610B613F618C
:04617C002A0EF66E83
:10618000100EF76E000EF86E00010900F550D26F88
:106190000900F550D36F03E1D26701D03DD009006B
:1061A000F550CD6F0900F550CE6F0900F550CF6F57
:1061B00009000900F550E96E0900F550EA6E090082
:1061C00009000900F550D06F0900F550D16F0900A2
:1061D0000900F6CFD4F0F7CFD5F0F8CFD6F0CDC088
:1061E000F6FFCEC0F7FFCFC0F8FF0001D05302E1A9
:1061F000D15307E00900F550EE6ED007F8E2D10761
:10620000F9D7D4C0F6FFD5C0F7FFD6C0F8FF00011C
:0A621000D207000ED35BBFD71200C7
:06621A00D9CFE6FFDACF48
:10622000E6FFFA0EE3CFD9FFFB0EE3CFDAFFFC0E59
:10623000E3CFE9FFFD0EE3CFEAFFE9CFF3FFEACFBB
:10624000F4FFF80EE35003E1F90EE35008E0F80E16
:10625000E30602E2F90EE306DECFEEFFF2D7FF0E11
:10626000E3CFDAFFE552FF0EE3CFD9FFE55212008C
:10627000FE0EE3CFE9FFFF0EE3CFEAFFE9CFF3FF26
:10628000EACFF4FFFB0EE35003E1FC0EE35009E01C
:10629000FB0EE30602E2FC0EE306FD0EE350EE6E9B
:0462A000F1D7120020
:0C62A40006500B02F3CF02F0F4CF03F021
:1062B0000C02F3500326000EF420046E06500D026B
:1062C000F3500426000EF420056E06500E02F35023
:1062D000052607500B02F3500326F4500422000E4B
:1062E000052207500C02F3500426F45005220750F3
:1062F0000D02F350052608500B02F3500426F4500B
:10630000052208500C02F350052609500B02F350E9
:04631000052612004C
:0C631400D9CFE6FFDACFE6FFE1CFD9FFDA
:10632000E2CFDAFFE652E652FC0EDBCF14F0FD0EB0
:10633000DBCF15F0060ED89014361536E804FBE1D5
:1063400014C0DEFF15C0DDFF010EDB50BB6EDF5059
:10635000E840E8403F0B300B146ECF0EBA14141017
:10636000BA6EE552E552E552E5CFDAFFE7CFD9FF45
:02637000120019
:0E637200D9CFE6FFDACFE6FFE1CFD9FFE2CFC9
:10638000DAFFE652E652FC0EDBCF14F0FD0EDBCF57
:1063900015F0060ED89014361536E804FBE114C04B
:1063A000DEFF15C0DDFF010EDB50BE6EDF50E840A2
:1063B000E8403F0B300B146ECF0EBD141410BD6EB1
:1063C000E552E552E552E5CFDAFFE7CFD9FF1200FB
:1063D000056A046A036A026A200EE76ED8900636E0
:1063E00007360836093602360336043605360B50B2
:1063F000025C0C5003580D5004580E50055809E328
:106400000B50025E0C50035A0D50045A0E50055AA0
:08641000062AE72EE4D7120072
:08641800D9CFE6FFDACFE6FF61
:10642000E1CFD9FFE2CFDAFFFD0EDB507E0BCD6E60
:10643000FD0EDBAC02D0CD8E01D0CD9ECF6ACE6AF0
:106440009E90DBAE02D09D8001D09D90CD80E55224
:0A645000E5CFDAFFE7CFD9FF120015
:06645A00D9CFE6FFDACF06
:10646000E6FFE1CFD9FFE2CFDAFFE652E652D6509F
:10647000DF6E010ED7CFDBFFDECF14F0DDCF15F0DE
:1064800014C0F3FF15C0F4FFE552E552E552E5CF25
:08649000DAFFE7CFD9FF12008B
:08649800056A046A036A180E8C
:1064A000E76ED890073608360936033604360536C7
:1064B0000C50035C0D5004580E50055807E30C5067
:1064C000035E0D50045A0E50055A072AE72EEAD7EC
:0264D0001200B8
:0E64D200D9CFE6FFDACFE6FFE1CFD9FFE2CF68
:1064E000DAFFE652E652FC0EDBCFDEFFDBCFDDFF4C
:1064F000010EDB50CF6EDF50CE6EE552E552E55215
:0A650000E5CFDAFFE7CFD9FF120064
:06650A00D9CFE6FFDACF55
:10651000E6FFE1CFD9FFE2CFDAFFE652E652FC0E0A
:10652000DBCFDEFFDBCFDDFF010EDB50D76EDF50B0
:10653000D66EE552E552E552E5CFDAFFE7CFD9FF57
:02654000120047
:0E654200D9CFE6FFDACFE6FFE1CFD9FFE2CFF7
:10655000DAFFFD0EDB507F0BD56ED76AD66AF29458
:10656000FD0EDBAE02D0F28A01D0F29AD58EE55252
:0A657000E5CFDAFFE7CFD9FF1200F4
:06657A00D9CFE6FFDACFE5
:10658000E6FFE1CFD9FFE2CFDAFFFD0EDB50FB0BD8
:10659000CA6ECC6A9E92FD0EDBAE02D09D8201D007
:1065A0009D92CA84E552E5CFDAFFE7CFD9FF12000A
:1065B000056A046A100EE76ED8900836093604366C
:1065C00005360D50045C0E50055805E30D50045E71
:0C65D0000E50055A082AE72EF0D71200E2
:0465DC00000EF36E4C
:1065E00000EE00F0080E01D81200EA6002D0EE6A58
:0C65F000FCD7F350E9601200EE6AFCD703
:0465FC0013EE00F0AA
:1066000023EE00F0F86A019CBEEC30F012EC33F09F
:08661000E7EC2AF0FBD71200B1
:06661800CD909D901200E0
:02661E00D59E07
:04662000F29A1200D8
:02662400120062
:0866260000000000000000006C
:02662E0000006A
:10663000000000000000000000000000000000005A
:0E66400000000000000000000000000000004C
:020000040030CA
:0100000024DB
:010001000EF0
:010002003FBE
:010003001EDE
:010005008179
:010006008178
:010008000FE8
:01000900C036
:01000A000FE6
:01000B00E014
:01000C000FE4
:01000D0040B2
:00000001FF
